:105B550001130000B30101020200000301FA040071
:105B6500FA0500030A0A5A0B001E0C00FA0D000381
:105B75000E00030F0164100096120132130AFA1485
:105B8500010215000017010A1801FA1905321A0158
:105B95000A1B01FA1C05321FFFFF20FFFF23011E10
:105BA5002400642A00FA2B00FA2C50782D003C2E94
:105BB50000462F001E3000643250783432FA350129
:105BC50064360164370150380A643C00643E003C89
:105BD5003F000040FFFF411450420A5A430AC8449F
:105BE50005324500B44600FA4701044802034C005B
:105BF500FA4EFFFF500404510596520A32530B46E4
:105C0500540A96560102570546580002590A465A43
:105C150032FA5B010A5C0A325E000A5F00FE61FF30
:105C2500FF64FFFF6600026701016A0A3C6B000022
:105C35006C32967300007400007801327901327E6F
:105C4500FFFF81FFFF84FFFF8500AF86000187000E
:105C5500FA89010A8A00009900009D0A969E0001B2
:105C65009FFFFFFAFAFA0000B301010202000003E8
:105C750001FA0400FA0500030A0A5A0B001E0C007B
:105C8500FA0D00030E00030F016410009612013295
:105C9500130AFA14010215000017010A1801FA196E
:105CA50005321A010A1B01FA1C05321FFFFF20FFEE
:105CB500FF23011E2400642A00FA2B00FA2C5078D9
:105CC5002D003C2E00462F001E30006432507834E3
:105CD50032FA350164360164370150380A643C00F4
:105CE500643E003C3F000040FFFF411450420A5A09
:105CF500430AC84405324500B44600FA4701024844
:105D050002024C00FA4EFFFF500404510596520A58
:105D150032530B46540A9656010157054658000161
:105D2500590A465A32FA5B010A5C0A325E000A5F7A
:105D350000FE61FFFF64FFFF6600026701016A0A5A
:105D45003C6B00006C3296730000740000780132E1
:105D55007901327EFFFF81FFFF84FFFF85FFFF860C
:105D6500FFFF87FFFF8901028A00009900009D0A55
:105D7500969E00019FFFFFFAFAFA0065006F007911
:105D85000083008D009700A100AC00B600C000CADA
:105D950000D400DE00E800F2005B0063006A0072D8
:105DA500007A008200890091009900A100A800B046
:105DB50000B800BF00C700CF00D600DF00E600EE48
:105DC50000F600400046004C00520059005F006597
:105DD500006B00710077007D00830089008F0095BE
:105DE500009C00A200A800AE00B400BA00C000C626
:0E5DF50000CC00D200D900DF00E500EB00F189
:1035E700900044E0D3940440149007B5E0FEA3E0B4
:1035F700FF905B57125F3CE493F59980129007B5F3
:10360700E0FEA3E0FF905C6B125F3CE493F59990BA
:1036170007B5E0FEA3E0FF905B55E493FC740193CC
:10362700FDEFB50507EEB50403754D009007B5121C
:103637005F232285F97285FA737E017F00E5731295
:103647005F15E5722FFF50010E8E598F5A900013A8
:10365700E0FCA3E0FDEF2DFDEE3CFC8C5B8D5C22D6
:1036670075A71085F97285FA737E017F00E57312DD
:103677005F15E5722FFF50010E8E598F5A9000D7B4
:10368700E0B40210AC2CAD2DEF2DFDEE3CFC8C5BB5
:103697008D5C8016AE59AF5A900013E0FCA3E0FD95
:1036A700EF2DFDEE3CFC8C5B8D5C22AE59AF5A745E
:1036B700B48E048F05FF125F058C5B8D5CAE59AF2E
:1036C7005A74B48E048F05FF125F308C598D5AE5FA
:1036D7005A4559601374B4C3955AFFE49559FE8E41
:1036E700598F5A785B125F6922900085E0B4010414
:1036F700C2138002D213900086E0B40104C2148082
:1037070002D2149000C3E075F0D2A4FFAEF0740AA1
:103717008E048F05FF125F059007ABECF0A3EDF069
:10372700A20D401674038C068D07125F15740112E3
:1037370000399007A9EEF0A3EFF07E017F0090001B
:1037470081E0125F159000C4E08E048F05FF125FC1
:1037570005740AFF125F058D5F9000CDE075F0D20A
:10376700A4FFAEF0740A8E048F05FF125F05900761
:10377700AFECF0A3EDF09000CFE060139000CFE046
:10378700F5F0741684FF7E00EF9007B9F080067499
:10379700649007B9F09000C5E0900069F090010FC0
:1037A700E0900053F090009EE0900055F09000C725
:1037B700E0900056F0900073E0900057F09000F909
:1037C700E090005CF074E3900068F09000AEE0B425
:1037D7000B0874E3900068F0805A9000AEE0B419CB
:1037E700129000C4E0905D6A12008CE49390006828
:1037F700F080419000AEE0B41E129000C4E0905DEE
:103807008812008CE493900068F080289000AEE066
:10381700B428129000C4E0905DB212008CE493903B
:103827000068F0800F9000AEE0B446089000A5E075
:10383700900068F090006CE0FE9000ABE0B50633B6
:1038470090006EE0FE9000C9E0B5062790006DE09D
:10385700FE9000D7E0B5061B900070E0FE90007E5A
:10386700E0B5060F90006FE0FE9000B9E06E7003C0
:103877000239BA900044E0C39405500874029000DE
:10388700FAF080149000D7E0600874089000FAF00E
:103897008006740A9000FAF090007EE0B401067486
:1038A700009000E4F090007EE0B4020674009000FF
:1038B700C9F090007EE0B4030674009000D6F09043
:1038C70000C9E0D39401401474189000FCF0740010
:1038D7009006C3F074009006C4F0800C740090004A
:1038E700FCF074189006C3F09000ABE06014741AF3
:1038F700900092F074009006CBF074009006CCF024
:10390700800C7400900092F0741A9006CBF090002F
:10391700ABE0B402147419900093F074009006C7DA
:10392700F074009006C8F0800C7400900093F07457
:10393700199006C7F09000D7E0700E74059006D76F
:10394700F074069006DBF0801874009006D7F074C8
:10395700009006D8F074009006DBF074009006DC47
:10396700F0D2299000ABE090006CF09000D7E09087
:10397700006DF09000C9E090006EF09000B9E09003
:10398700006FF090007EE0900070F090007EE09075
:103997000054F09000B9E0900058F09000D7E09004
:1039A7000059F09000ABE090005AF09000C9E09009
:1039B700005BF09000E1E0B4011790001F740FF076
:1039C700A374FFF0900021E4F0A3F074029000E1EB
:1039D700F09000E1E0B40341900021E0FEA3E0FF96
:1039E70090001FE0FCA3E0FD125F617410125F15E9
:1039F7007408120039EF900065F0EF700674FF90BD
:103A07000065F074009000E1F0900020E0900066FF
:103A1700F090001FE0900067F0900072E09000398E
:103A2700F0900039E00490003AF090003AE0D39427
:103A370002400B90003AE0C3940290003AF07550B0
:103A4700019000B8E090003BF090003BE0D3940277
:103A5700400F90003BE0C3940290003BF0D22380DC
:103A670002C22390003BE0D39401400890003C74CD
:103A770001F08006740290003CF022C293C294C207
:103A870091C292C287C290E5B554EFF5B5E5B5543A
:103A9700DFF5B5C296C295C2A0C297C2A2C2A1E580
:103AA700B554BFF5B5E5B5547FF5B5E5B554FBF5A8
:103AB700B5C215755D469000BBE07005756C028058
:103AC70003756C0375540075530090000874FFF07C
:103AD700A374DCF0C21AC21C74C8900035F074C815
:103AE700900037F0755200755100C20D754600E51C
:103AF7006EB40903756E00756200900015E4F0A3BB
:103B0700F0756F10C218C2199007ABE0FEA3E0FF73
:103B17007403125F1574011200399007A9EEF0A320
:103B2700EFF0C20275560075550090000CE4F0A343
:103B3700F0C22A75580075570090007DE075F03285
:103B4700A4FDACF090001DECF0A3EDF090003374F1
:103B570075F0A37430F0C20EC20FC23A2285F97213
:103B670085FA737E017F00E573125F15E5722FFFFB
:103B770050010E8E598F5AAC5BAD5CEF2DFDEE3CBC
:103B8700FC8C5B8D5CD293D294E55CF5FBE55BF531
:103B9700FCE55CF5E9E55BF5EA9000B9E0B40314F0
:103BA700D291D292E55CF5EBE55BF5ECE55CF5EDE2
:103BB700E55BF5EE2275A71085F97285FA737E012C
:103BC7007F00E573125F15E5722FFF50010E8E59C6
:103BD7008F5A7E017F769000F6E0125F15AC59ADE3
:103BE7005AED2FFFEC3EFE8E5B8F5CE55CF5FDE545
:103BF7005BF5FE900069E4F075A700741290004031
:103C0700F02285F97285FA737E017F00E573125FF2
:103C170015E5722FFF50010E8E598F5A9007ABE0B2
:103C2700FCA3E0FDEF2DFDEE3CFC8C5B8D5CE55CC1
:103C3700F5FDE55BF5FE220563229000B9E0B403CC
:103C4700539000D7E0B4012EA2D8B34004C293C268
:103C570087A2D9B34004C294C290A2DAB34008C283
:103C670091E5B554EFF5B5A2DBB34008C292E5B5CF
:103C770054DFF5B5801CA2D8B34002C293A2D9B3D2
:103C87004002C294A2DAB34002C291A2DBB340025F
:103C9700C292801EA2D8B3400AC2939000D7E060B8
:103CA70002C287A2D9B3400AC2949000D7E060024B
:103CB700C290A2DCB34004C296C29575D840228553
:103CC700A77175A710A2D8B34002C287A2D9B34083
:103CD70002C290A2DAB34006E5B554EFF5B5A2DB10
:103CE700B34006E5B554DFF5B5A2DCB34008900054
:103CF700C5E0900069F075D8408571A7229000470C
:103D0700E4936406600280FE74C89007B1F8E4F09B
:103D1700E8A3F075B50075840175A70075FFA0903D
:103D2700003DE4F075C91075A70F75A1C775A70009
:103D370075D90075CE0C75A70F75F1FE75F2FF7575
:103D4700F30775F47875A4BA75A5FF75A60775AE60
:103D57000075AFFF75D48175D5FF75D6FF75D7FF91
:103D670075A70075A20175A14775F80975D8007583
:103D7700D90475DA0975DB0975DC0975DD0975DEA6
:103D87000975D84075A71075D80075D90475DA0973
:103D970075DB0975DC0975DD0975DE0975D84075B0
:103DA700A70075E60875E71075BC0175BE0475BDFB
:103DB7006C75BE0775BDA075BE0875BD0175BC00E5
:103DC70075BB1875BC2075BA0875E88075D1137571
:103DD700A70F75E10575E20075C740123A8275971E
:103DE70000759780740A125EF57597C0E5975420A1
:103DF700700280F8758F0275A700D2AF75980075AD
:103E0700A90C75A70F75AB4375ADFB75AC1E75A7F0
:103E17001075C91875CA0075CB0075C80475A70059
:103E2700758912758E04758C00758A00C2A9D28CAB
:103E3700758D00758B00D2ABD28E75EF0675D944A0
:103E4700C29974C8F5097508001200E375B5001228
:103E570004E374639007B1F8E4F0E8A3F012036F8A
:103E670074C89007B1F8E4F0E8A3F07464F5097535
:103E770008001200E3900054E090007EF0C220900A
:103E8700007EE0D394034006740090007EF090001B
:103E97007EE090576DF82828738028A2B44002D29C
:103EA70020802075A70F75F30F75A700A2A3400206
:103EB700D220800F75A70F75F31775A700A2A4402E
:033EC70002D22004
:0C576D00023EA0023EA2023EAA023EBB89
:103ECA00A220B34066757208E572D3940E5020E5BD
:103EDA00729007B1F8E4F0E8A3F012023E7464F5B8
:103EEA00097508001200E37872740126F650D97435
:103EFA00029000BAF090007EE0D39403400674006A
:103F0A0090007EF090007EE0905779F82828738020
:103F1A001674009000E4F0800E74009000C9F080DE
:073F2A000674009000D6F0C0
:0C577900023F19023F1B023F23023F2B9E
:103F3100D21F8064757201E572D394075020E57237
:103F41009007B1F8E4F0E8A3F012023E7464F509B9
:103F51007508001200E37872740126F650D97401D5
:103F61009000BAF090007EE0D39403400674009074
:103F7100007EF090007EE0905785F8282873801627
:103F810074009000E4F0800E74009000C9F0800687
:063F910074009000D6F060
:0C578500023F7F023F81023F89023F91FA
:103F9700C21F900053E090010FF0900054E0900092
:103FA7007EF0900055E090009EF0900056E0900063
:103FB700C7F0900057E0900073F0900058E0900031
:103FC700B9F0900059E09000D7F090005AE09000C7
:103FD700ABF090005BE09000C9F090005CE09000CF
:103FE700F9F09000C4E07006740A9000C4F09000E5
:103FF700A5E0700674E39000A5F09000ABE0049094
:10400700006CF01236F0E5B54401F5B57406900082
:1040170042F07401900043F07403900045F074057A
:10402700900046F07427900047F07405900048F020
:10403700900044E0B404067404900048F0740090C3
:104047000049F0740090004EF0740090004FF07437
:1040570001900050F07400900051F074FF900052EE
:10406700F0744E900148F07469900149F0747390B0
:10407700014AF0747390014BF0746190014CF07435
:104087006E90014DF0742090014EF0743490014F02
:10409700F07443900150F07479900151F0746C9072
:1040A7000152F07420900153F07420900154F07481
:1040B70020900155F07420900156F09000E0E090B8
:1040C7000065F0900097E0900066F0900098E0900F
:1040D7000067F0A2B6B39211A2B3B39212A2A4B32F
:1040E7009226A2B4B39227A2A3B39228900061E4C8
:1040F700F0756E00743A900771F074FD900772F0D6
:10410700900062E4F09007ABE0FEA3E0FF740312B7
:104117005F1574011200399007A9EEF0A3EFF0754F
:104127006D01900040E4F0C225756200C216D217F7
:10413700C202757000C22CD203C22DD204C22ED285
:1041470005C22FD206C230D207C231D208C232D23C
:1041570009C233D20AC234D20BC235D20CC221C231
:1041670022C223C224C22912009E755E00756A000E
:104177007560007564327565007566007567007552
:104187006800756900900015E4F0A3F0756B00D224
:10419700B2D2A4D2B0D2B1D2A3D2A7D2A6D2A5D23C
:1041A700B790007DE0D394FA400674FA90007DF052
:1041B7007E017F00900067E0125F15900066E02F98
:1041C700FF50010E90001FEEF0A3EFF0EFD394FF26
:1041D700EE940F400790001FE4F0A3F0900065E015
:1041E700700674FF900065F074009000A4F09000D2
:1041F700BAE0D39402400674019000BAF09000BB75
:10420700E07005756C028003756C039000BCE0D309
:104217009401400674009000BCF09000C2E0C39483
:104227000A5006740A9000C2F09000CCE070067441
:10423700019000CCF09000CCE0B4FF0674FE900033
:10424700CCF09000D3E0D394FE400674FE9000D3E8
:10425700F09000F9E0D39402400674019000F9F061
:1042670090010FE0D394014006740190010FF074A0
:10427700019000D9F074019000DAF074009000E129
:10428700F074009000FDF07400900101F074299023
:1042970006B7F0742A9006BBF074179006BFF07447
:1042A7001B9006CFF0741C9006D3F0D29C9000AC04
:1042B700E0D39404400674049000ACF09000DEE074
:1042C700D39404400674049000DEF0E56FD3941095
:1042D7004003756F109006B8E0D3940C4006740045
:1042E7009006B8F09006BCE0D3940C40067400909A
:1042F70006BCF09006C0E0D3940C4006740090060C
:10430700C0F09006C4E0D3940C400674009006C435
:10431700F09006C8E0D3940C400674009006C8F0ED
:104327009006CCE0D3940C400674009006CCF09035
:1043370006D0E0D3940C400674009006D0F09006A7
:10434700D4E0D3940C400674009006D4F09006D8BD
:10435700E0D3940C400674009006D8F09006DCE099
:10436700D3940C400674009006DCF0D2EC75CF01B4
:10437700A298B34005C298120616E54D6006A299A9
:10438700B3B340028005C299120AB4E54E640160D6
:1043970005E54EB4040280D5C28E7E087F00E56332
:1043A700125F15E58D75F008A4FDACF0EF2DFDEE5D
:1043B7003CFCE58B75F02084FF7E00ED2FFFEC3E83
:1043C700FE8E538F54D28E90009EE0605C90001753
:1043D700125F23900017E0FCA3E0FD900019E0FABC
:1043E700A3E0FBEDB50342ECB5023EB21EA20DB34E
:1043F700401975E700A21EB34008E5B54404F5B5BA
:104407008006E5B554FBF5B575E710900019E0FE99
:10441700A3E0FF90001BE0FCA3E0FDEF2DFDEE3CC9
:10442700FC900019ECF0A3EDF09000ABE060099070
:1044370000ABE0C394034002806F1229C0A20DB302
:104447005009900061E0C3940740028006900095F0
:10445700E0F545E54575F005A4FFAEF09007B3EE2E
:10446700F0A3EFF0900082E0C395604007E55EC3DC
:10447700955F50079007B3E4F0A3F0AE2EAF2F90EF
:1044870007B3E0FCA3E0FDEFD39DEE9C4004C2A17F
:10449700800B900061E0C3940A5002D2A19000AB58
:1044A700E0B40205A2A1B392A29000ABE0B4031C52
:1044B700122ADBAE2EAF2F9007B3E0FCA3E0FDEF8F
:1044C700D39DEE9C4004D2A18002C2A1A2B63011B6
:1044D70001B35003024A34A2B6301101B3500302AC
:1044E7004A34A2B6301301B3500302484C756D002D
:1044F700055DA20EB350030245B2E56CB4032EA2CC
:104507002AB34022E55DB40503756C01E55DC394EC
:104517000550069000407401F0E55DD39405400610
:104527007402900040F0755D01D22A805AE56CB4A0
:104537000206756C01755D03E55DB40305755D01E4
:104547008045900040E07030E55DC39403500690CD
:1045570000407401F0E55DD39403400674029000B7
:1045670040F0E55DC394035002D225E55DD3940383
:104577004002D225C296C2959000BBE0B401051255
:104587003A828003755D01C20EC20FA2239222A256
:10459700B4B34002C227A2A4B34002C226A2A3B367
:1045A7004002C228A225B34002C225E56CC394038A
:1045B7005006E55D640360028016B222755D01A2B4
:1045C7000F4004B20F80097405900040F0123A8240
:1045D7009000B9E0B4030890003BE0655D6002809D
:1045E7000BA222B34004D2248002C224E55DB402A8
:1045F7004990009EE06043900017E0FEA3E0FF9023
:10460700009EE08E048F05FF125F0574018C068DF6
:104617000712003990001BEEF0A3EFF090001BE0AB
:10462700F8A3E0900019C8F0A3C8F0900017E4F0D1
:10463700A3F0C21EE5B554FBF5B5AE57AF58AC5362
:10464700AD54EF2DFDEE3CFC8C578D58AE53AF5457
:10465700EFD39DEE9C401190000FE0FAA3E0FBEB37
:10466700C394E8EA94034002800690000F125F2388
:10467700900008E553F0A3E554F090000AE553F0E5
:10468700A3E554F0AE53AF5474128E048F05FF1296
:104697005F058C558D56C28E758D00758B007563C1
:1046A70000755401755300D28E900008E0FEA3E018
:1046B700FFEF4E600B7C7E7D63125E038E518F523F
:1046C700AE51AF527428BE00039F5010E5622FFF12
:1046D70050010E74011200398E518F52855262902B
:1046E70000C2E0A851B8000DD395524008E552909A
:1046F700003FF080099000C2E01490003FF0E56CA5
:1047070060067552007551009000ABE060031220FF
:104717002BE56EB40903756E00A216B35006A215F9
:10472700B3B340030247D3900077E0B4017390001E
:10473700F9E0B40214120C5590006AE075F0BEA4BB
:10474700FFAEF08E5B8F5C8056E56675F00A84FFDE
:104757007E00900571125F3CE0F55A755900AE591D
:10476700AF5A90009CE0125F1574648E048F05FFAA
:10477700125F058C5B8D5CE55C90000EF0AE59AF67
:104787005A900075E0125F1574648E048F05FF124E
:104797005F0574BE8C068D07125F158E5B8F5C807C
:1047A70017900075E075F0BEA4FFAEF08E5B8F5CCE
:1047B70090009CE090000EF0E560C394CC5006900A
:1047C7000075E070028003123B64D216E56CB401F9
:1047D70006A215B3B340028009756F0190004174BA
:1047E70001F0E56C705A9000BEE0600D900069E042
:1047F700A851B800069552400280299000BEE0B447
:104807000208756F03756B00800CC200756B009012
:104817000015E4F0A3F0900069E0600674099000C9
:1048270040F0801CE55DB40109756F01900041748B
:1048370001F0E55DB40209756F017402900041F063
:10484700A213B39211A213B330B601B35003024AB5
:1048570034756D01E5B54401F5B57407900061F055
:10486700A2139211E55DD394474014D215E55DD3A9
:10487700944B400B7405900040F0D225755D46902F
:1048870000C6E0B40107E569C39414400280091229
:104897003A827413900040F0A215B3B350189000F9
:1048A70033E0FEA3E0FF7402125F15AC53AD54EF83
:1048B700C39DEE9C40028002D20E900033E553F078
:1048C700A3E554F0A22C300301B3501D75E700A2F5
:1048D7002CB34008E5B54408F5B58006E5B554F7AF
:1048E700F5B575E710A22C9203A22D300401B35041
:1048F7001D75E700A22DB34008E5B54402F5B58064
:1049070006E5B554FDF5B575E710A22D9204A22E64
:10491700300501B3500FA22EB34004D2A08002C2CB
:10492700A0A22E9205A22F300601B3500FA22FB3DB
:104937004004D2978002C297A22F9206A230300776
:1049470001B3500FA230B34004D2A28002C2A2A288
:10495700309207A231300801B3500FA231B340049F
:10496700D2A18002C2A1A2319208A232300901B3BA
:10497700501D75E700A232B34008E5B54440F5B5D0
:104987008006E5B554BFF5B575E710A2329209A2C6
:1049970033300A01B3501D75E700A233B34008E571
:1049A700B54480F5B58006E5B5547FF5B575E710D4
:1049B700A233920AA234300B01B3500FA234B34092
:1049C70004D2878002C287A234920BA235300C0131
:1049D700B3500FA235B34004D2908002C290A235E3
:1049E700920CE569C394415009740E900040F0128F
:1049F7003A82900048E0FE900044E004C39E4009DC
:104A0700900044E0D39406400974FB900040F012F4
:104A17003A8290004DE0601590004DE0FE9000470F
:104A2700E06E600974FE900040F0123A82A225B34E
:104A37004004C296C2959000F6E0600CAE51AF52AA
:104A47007414BE00059F4002804890007EE0905796
:104A570091F8282873803BA2B4B35005A227B3402E
:104A6700028005123BBCD2278028A2A3B35005A21F
:104A770028B340028005123BBCD2288015A2A4B3FC
:104A87005005A226B340028005123BBCD226800205
:024A970080009D
:10579100024A5C024A5E024A71024A84024A970244
:0257A1004A9923
:104A9900A218B3B3500890003BE0655D6003024B78
:104AA90078A201B35006A200B3B34003024B74903D
:104AB90000B9E0B403028003024B49A20DB3406779
:104AC900A224B3402D12363AE55CF5FBE55BF5FC13
:104AD900D293A202B34002D2879000D7E0B4021069
:104AE900123667E55CF5FBE55BF5FC75A700D28737
:104AF900803312363AE55CF5EBE55BF5ECD291A231
:104B090002B34006E5B54410F5B59000D7E0B4020C
:104B190014123667E55CF5EBE55BF5EC75A700E586
:104B2900B54410F5B5801712363AE55CF5FBE55B3F
:104B3900F5FCE55CF5EBE55BF5ECD293D291802BC6
:104B490012363AE55CF5FBE55BF5FCD293A202B3BC
:104B59004002D2879000D7E0B40210123667E55CB4
:104B6900F5FBE55BF5FC75A700D287C218D219A23F
:104B790019B3B3500890003CE0655D6003024C57DF
:104B8900A201B35006A200B3B34003024C539000F4
:104B9900B9E0B403028003024C28A20DB34067A216
:104BA90024B3402D12363AE55CF5E9E55BF5EAD226
:104BB90094A202B34002D2909000D7E0B40210123E
:104BC9003667E55CF5E9E55BF5EA75A700D2908003
:104BD9003312363AE55CF5EDE55BF5EED292A202C9
:104BE900B34006E5B54420F5B59000D7E0B402140A
:104BF900123667E55CF5EDE55BF5EE75A700E5B501
:104C09004420F5B5801712363AE55CF5E9E55BF520
:104C1900EAE55CF5EDE55BF5EED294D292802B12D4
:104C2900363AE55CF5E9E55BF5EAD294A202B340D0
:104C390002D2909000D7E0B40210123667E55CF515
:104C4900E9E55BF5EA75A700D290D218C219E56FBC
:0E4C59009057A3F82828730250E09000DEE088
:0657A300024C60024C63A1
:104C67009057D6F8282873121B078012121B07804B
:0E4C77000D121B918008121C3D8003121C3D83
:0F57D600024C6E024C73024C78024C7D024C82E6
:104C8500756F020250E0121D69121E80A23AB340F0
:104C95000C9000A0E0F56B7410900040F09000714E
:104CA500E0256BF5349007A9E0FEA3E0FF740A1236
:104CB5005F1590000AE0FCA3E0FD74098F02FF1266
:104CC5005F058D078C038E048A058B06125E0390A3
:104CD50007ADEEF0A3EFF09000C7E0B401087478DB
:104CE500BE00059F4002800D74789007ADF8E4F092
:104CF500E8A3F0801B9007ADE0FEA3E0FF74F0BED3
:104D050000039F500B74F09007ADF8E4F0E8A3F0B2
:104D1500E53470037534019007ADE0FEA3E0FFE5CF
:104D2500342FFF50010E9007ADEEF0A3EFF0756F35
:054D350003900041E0C5
:0357A900024C8B24
:104D3A009057E5F82828738010A23B4003756F0A44
:094D4A008007A23B4003756F0BCA
:0957E500024D41024D43024D4CFE
:104D53000250E09006B8E060031221149000F7E0DF
:104D6300B401149000F8E0A851B80004955250071C
:104D7300E55EC3955F40028003024E009000ACE005
:104D8300D39402403F900080E02403A851B800046C
:104D930095525009900082E0D3956050028008D26A
:104DA300017408900040F0900080E0A851B800051D
:104DB300D39552500B900082E02403C395605002B8
:104DC300C2018039900080E02403A851B800049503
:104DD300525007E55EC3955F40028008D201740814
:104DE300900040F0900080E0A851B80005D39552A0
:104DF3005009E55F240FC3955E5002C2019000C6BF
:104E0300E07007E569C3941440028002D201A20155
:104E13004005756F04800A756F10900015E4F0A3C8
:104E2300F0A20DB34029E56675F00A84FF7E009079
:104E33000571125F3CE0C394695005122060800F36
:104E43009007ABE0F8A3E09007A9C8F0A3C8F0026D
:064E530050E09000ACE00D
:0657AC00024D56024E55AD
:104E59009057EEF8282873120D3F8012120D3F80EB
:0E4E69000D120EED8008120F9F8003120F9F96
:0F57EE00024E60024E65024E6A024E6F024E740A
:104E77009006BCE060031221F0756F050250E01246
:104E870010AB756F069006C0E060031222E0900633
:104E9700C4E060031223BC0250E090000EE06006FD
:104EA700A20DB3B34002801D90000EE02529FFAE8E
:104EB7002850010E8E288F29E55DD3940150069066
:104EC700000EE014F01212F1756F079006C8E0604B
:104ED700031224989006CCE060031225740250E078
:104EE7009000F9E0B40203120CCD12154E756F084D
:104EF7009006D0E060031226509006D4E0600312BB
:104F0700272C0250E012190AA218B35005A219B3B0
:104F170040028004D218D219756F109006D8E0604D
:104F2700031228089006DCE060031228E40250E030
:104F37000250E0900036E0C394465008C29674468B
:104F4700900036F085345A755900900039E0F572B3
:104F57001236B2E55C900036F0900004E559F0A3F4
:104F6700E55AF0C21B900072E0FE900036E0C39E47
:104F77005012900072E0FE900036E0F4042E90008C
:104F870036F08012900072E02402FE900036E0F4C2
:104F9700042E900036F09007ADE0F559A3E0F55ADE
:104FA700900039E0F5721236B2E55C900035F0906A
:104FB7000000E559F0A3E55AF0C21A900072E0FE2E
:104FC700900035E0C39E5012900072E0FE900035CD
:104FD700E0F4042E900035F08012900072E0240275
:104FE700FE900035E0F4042E900035F0E56CB40136
:104FF70005756F0B8003756F030250E0900038E072
:10500700C3944650139000C7E0B40104C2968002CF
:10501700C2957446900038F085345A75590090004F
:105027003AE0F5721236B2E55C900038F09000066F
:10503700E559F0A3E55AF0C21D900072E004FE9016
:105047000038E0C39E5013900072E004FE900038D1
:10505700E0F4042E900038F08012900072E02403F0
:10506700FE900038E0F4042E900038F09007ADE091
:10507700F559A3E0F55A90003AE0F5721236B2E519
:105087005C900037F0900002E559F0A3E55AF0C2B2
:105097001C900072E004FE900037E0C39E5013900E
:1050A7000072E004FE900037E0F4042E900037F021
:1050B7008012900072E02403FE900037E0F4042E83
:1050C700900037F0E56CB40103756C00756F0380D1
:0950D700088006800480028000BC
:1057B200024E86024EA1024EE7024F0C024F370202
:1057C2004F3A0250030250D80250DA0250DC025023
:0457D200DE0250E0C3
:1050E000900035E0B55D02800302517BA21A406B4F
:1050F000900000E0FEA3E0FFEF4E605DAC51AD52CA
:10510000740ABC0033D39D402FAA55AB5674058A50
:10511000048B05FF125F058D068C07900000E0FCF4
:10512000A3E0FDCFCECF120003740112003990002E
:1051300000EEF0A3EFF08021AE55AF56900000E0F6
:10514000FCA3E0FD120003740A8E048F05FF125FBA
:1051500005900000ECF0A3EDF0D21AAE53AF5490DE
:105160000000E0FCA3E0FDEFC39DEE9C400D123C6F
:1051700009D296C21A74C8900035F0A21AB3B3507F
:1051800007900035E0B55D02800D123C09D296749F
:10519000C8900035F0C21A900036E0B55D02800379
:1051A00002522FA21B406B900004E0FEA3E0FFEF31
:1051B0004E605DAC51AD52740ABC0033D39D402F9C
:1051C000AA55AB5674058A048B05FF125F058D0640
:1051D0008C07900004E0FCA3E0FDCFCECF120003CB
:1051E0007401120039900004EEF0A3EFF08021AEBC
:1051F00055AF56900004E0FCA3E0FD120003740AD2
:105200008E048F05FF125F05900004ECF0A3EDF013
:10521000D21BAE53AF54900004E0FCA3E0FDEFC3FB
:105220009DEE9C400AC2967446900036F0C21BA2C6
:105230001BB3B35007900036E0B55D02800AC296FA
:105240007446900036F0C21B900037E0B55D0280D6
:10525000030252EEA21C406B900002E0FEA3E0FFAE
:10526000EF4E605DAC51AD52740ABC0033D39D402B
:105270002FAA55AB5674058A048B05FF125F058D66
:10528000068C07900002E0FCA3E0FDCFCECF120019
:10529000037401120039900002EEF0A3EFF08021B8
:1052A000AE55AF56900002E0FCA3E0FD120003747F
:1052B0000A8E048F05FF125F05900002ECF0A3ED4B
:1052C000F0D21CAE53AF54900002E0FCA3E0FDEF1F
:1052D000C39DEE9C4018123C099000C7E0B4010445
:1052E000D2968002D295C21C74C8900037F0A21CDE
:1052F000B3B35007900037E0B55D028018123C0947
:105300009000C7E0B40104D2968002D29574C89090
:105310000037F0C21C900038E0B55D0280030253F4
:10532000B8A21D406B900006E0FEA3E0FFEF4E60C8
:105330005DAC51AD52740ABC0033D39D402FAA55C9
:10534000AB5674058A048B05FF125F058D068C072A
:10535000900006E0FCA3E0FDCFCECF120003740165
:10536000120039900006EEF0A3EFF08021AE55AFA9
:1053700056900006E0FCA3E0FD120003740A8E04C0
:105380008F05FF125F05900006ECF0A3EDF0D21D33
:10539000AE53AF54900006E0FCA3E0FDEFC39DEEDA
:1053A0009C40159000C7E0B40104C2968002C295EB
:1053B0007446900038F0C21DA21DB3B35007900090
:1053C00038E0B55D0280159000C7E0B40104C296D4
:1053D0008002C2957446900038F0C21D9000C9E06A
:1053E000B4020280030254F8900063E0D395655044
:1053F00064900063E0F4042565FE9000CCE08E002C
:10540000F5F0E884FF7E008F72EFC39410500CEF2C
:105410008572F0A4FDACF08D7280037572FF900070
:1054200063E0D39572400B900063E0C39572F57012
:1054300080037570009000E7E0D3957040069000FF
:10544000E7E0F5709000E8E0C3957050069000E842
:10545000E0F5708071900063E0C39565FE9000CC2C
:10546000E08E00F5F0E884FF7E008F72EFC39410A9
:10547000500CEF8572F0A4FDACF08D728003757254
:10548000FF85725A755900900063E0255AFFAE59A6
:1054900050010E8E598F5A74FFBE0009D39F4005EC
:1054A000855A7080037570FF9000E7E0D3957040D7
:1054B000069000E7E0F5709000E8E0C395705006B4
:1054C0009000E8E0F570A20DB3B3500D900064E0D9
:1054D000FE9000D4E0D39E5002800A7407900040F2
:1054E000F0C297801375A710E5CDC395704004C234
:1054F000978002D29775A700E56EC39409500AA25F
:10550000EDB34005C2ED122C7AAE53AF5474B8C35C
:105510009F74889E400C900062E0C3945A4003023E
:10552000576AA215B34009123A827406900040F0FF
:10553000A220B34008E5B54404F5B58006E5B554AE
:10554000FBF5B5A217B3500EE560D394334007E5E1
:1055500060C394CC4002802FE5B54401F5B57407D3
:10556000900061F0900075E075F0BEA4FFAEF08E83
:105570005B8F5C7402BE000AD39F4006755C0275A7
:105580005B00123B64D217900062E0D394014007A5
:10559000E560C3941A40028002C2179006B8E0602A
:1055A00003122114A22C300301B35017A22CB340D4
:1055B00008E5B54408F5B58006E5B554F7F5B5A29C
:1055C0002C92039006BCE060031221F0A22D30045F
:1055D00001B35017A22DB34008E5B54402F5B580DC
:1055E00006E5B554FDF5B5A22D92049006C0E06025
:1055F000031222E0A22E300501B3500FA22EB340B9
:1056000004D2A08002C2A0A22E92059006C4E0603F
:10561000031223BCA22F300601B3500FA22FB340B8
:1056200004D2978002C297A22F92069006C8E0602B
:1056300003122498A230300701B3500FA230B340B8
:1056400004D2A28002C2A2A23092079006CCE060EF
:1056500003122574A231300801B3500FA231B340B8
:1056600004D2A18002C2A1A23192089006D0E060CB
:1056700003122650A232300901B35017A232B340B0
:1056800008E5B54440F5B58006E5B554BFF5B5A2CB
:105690003292099006D4E0600312272CA233300A1C
:1056A00001B35017A233B34008E5B54480F5B58087
:1056B00006E5B5547FF5B5A233920A9006D8E060AE
:1056C00003122808A234300B01B3500FA234B340A8
:1056D00004D2878002C287A234920B9006DCE0607D
:1056E000031228E4A235300C01B3500FA235B340A9
:1056F00004D2908002C290A235920C900062E0C366
:10570000945A5010E56EB40909900062E004F075F7
:105710006E00803BE56EB40903756E00755400752C
:105720005300758D00758B00756300900061E0C3B8
:10573000940A5008900061E004F08006740A90001A
:1057400061F0900061E0B40A06E5B554FEF5B5904D
:105750000062E0D394014007E569C39441400280B0
:0D57600009740E900040F0123A820243746A
:1057FD000000010001400160018001A001C001E035
:10580D0002000300039603B603D603F4040005005B
:10581D000512052405360548055A056C057E0590CB
:10582D0005A805C005DE0600061406280646066E08
:10583D0006AE00FF013F015F017F019F01BF01DF48
:10584D0001FF02FF039503B503D503F303FF04FF27
:10585D0005110523053505470559056B057D058F93
:10586D0005A705BF05DD05F1061306270645066DDF
:10587D0006AD06ED0FAA0FA50F9F0F9A0F940F8D72
:10588D000F870F800F780F710F680F600F570F4E36
:10589D000F450F3B0F300F250F1A0F0E0F020EF590
:1058AD000EE80EDB0ECC0EBE0EAE0E9F0E8E0E7DD6
:1058BD000E6C0E5A0E470E340E200E0C0DF70DE227
:1058CD000DCB0DB50D9D0D850D6D0D540D3A0D20A6
:1058DD000D050CE90CCE0CB10C940C760C580C3A51
:1058ED000C1B0BFB0BDB0BBB0B9A0B790B570B3507
:1058FD000B130AF10ACE0AAB0A870A640A400A1C86
:10590D0009F809D409B0098C09670943091F08FB77
:10591D0008D608B2088E086A0846082307FF07DC78
:10592D0007B9079607730751072F070D06EC06CA2F
:10593D0006AA068906690649062A060A05EC05CD5A
:10594D0005B0059205750558053C0520050504EAC9
:10595D0004CF04B5049C0482046904510439042263
:10596D00040B03F403DE03C803B2039D038903751F
:10597D000361034D033B03280316030402F202E106
:10598D0002D102C002B002A002910282027302652E
:10599D0002570249023C022F02220216020901FDA2
:1059AD0001F201E601DB01D001C601BB01B101A786
:1059BD00019D0194018B01820179017001680160E3
:1059CD00015801500148014101390132012B0125D6
:1059DD00011E01180111010B010500FF00FA0FA6B0
:1059ED000FA00F990F920F8B0F840F7C0F740F6BFD
:1059FD000F620F580F4E0F430F380F2C0F1F0F1242
:105A0D000F050EF70EE80ED80EC80EB70EA50E93A5
:105A1D000E800E6C0E580E420E2C0E150DFD0DE463
:105A2D000DCB0DB10D950D790D5D0D3F0D200D01BA
:105A3D000CE10CC00C9E0C7C0C590C350C100BEAB7
:105A4D000BC40B9E0B760B4F0B260AFD0AD40AAA2C
:105A5D000A800A550A2A09FF09D409A8097C0950A8
:105A6D00092508F908CD08A10875084A081E07F38D
:105A7D0007C8079D07730749072006F706CE06A638
:105A8D00067E06570630060A05E405BF059B057719
:105A9D0005540532051004EF04CE04AE048F0471D5
:105AAD0004530435041903FD03E203C703AD039446
:105ABD00037B0363034B0334031E030802F302DE6F
:105ACD0002CA02B602A30291027F026D025C024C71
:105ADD00023C022C021D020E020001F201E401D76C
:105AED0001CA01BE01B101A6019A018F0185017A9A
:105AFD0001700166015D0153014A01410139013116
:105B0D000129012101190112010B010400FD00F70A
:105B1D0000F000EA00E400DE00D900D300CE00C999
:105B2D0000C400BF00BA00B500B100AD00A800A4CC
:105B3D0000A0009C009900950091008E008A0087BE
:085B4D0000840081007E007B52
:10009E007547009007B5E4F0A3F075310075300098
:1000AE00754D00754E00C237D23874FE9007BFF8FA
:1000BE00E4F0E8A3F074FE9007C1F8E4F0E8A3F0D2
:1000CE00745A9007C3F0745A9007C4F0D239C22BF9
:1000DE00C23BC23622750B00750A00AE0AAF0BACDE
:1000EE0008AD09EDC39FEC9E401674FF125EF575C8
:1000FE00CF01780B740126F6500418E436F650DB67
:10010E002290003DE0B4AA1C900771E0B43C15901B
:10011E0007B1E0FEA3E0FFEF4E6009741EBE0004BF
:10012E00D39F500302023D755C00755B0075F809A4
:10013E009007B1E0FEA3E0FF74076F4E6006740EE9
:10014E006F4E7006743A900771F09007B1E0FEA3FF
:10015E00E0FF7408BE001ED39F401A7E017F0890F8
:10016E0007B1E0FCA3E0FD1DBDFF011C1200038ED4
:10017E00598F5A801F9007B1E0FEA3E0FF7408125A
:10018E005F598F048E057E017F08CDCCCD12000302
:10019E008E598F5AAE5BAF5C740CD39F74019E5018
:1001AE0003020238A2F9B3407EE55C455B7003752D
:1001BE00A382AE5BAF5C74016F4E700375A300AE8D
:1001CE005BAF5C74026F4E700D9007B2E075F0027B
:1001DE00A4FDACF08DA3AE5BAF5C74036F4E7003E9
:1001EE0075A300AE5BAF5C7403BE00039F5013ACEF
:1001FE0059AD5AED2FFFEC3EFE90006D125F3CE0C4
:10020E00F5A3AE5BAF5CEFB40B09EEB4010574144D
:10021E00125EF5AE5BAF5CEFB40B07EEB401037587
:10022E00F80D785B125F690201A290003DE4F022A6
:10023E00755C00755B0075F8099007B1E0FEA3E0F0
:10024E00FF7408BE001ED39F401A7E017F089007E0
:10025E00B1E0FCA3E0FD1DBDFF011C1200038E5991
:10026E008F5A801F9007B1E0FEA3E0FF7408125F63
:10027E00598F048E057E017F08CDCCCD1200038EE2
:10028E00598F5AAE5BAF5C7411D39F74019E5003AD
:10029E0002036EA2F9B3500302036BE55C455B707B
:1002AE000375A3D2AE5BAF5C74016F4E700375A382
:1002BE0000AE5BAF5C74026F4E700D9007B2E075CE
:1002CE00F002A4FDACF08DA3AE5BAF5C74036F4E79
:1002DE00700375A300AE5BAF5C74046F4E70037554
:1002EE00A300AE5BAF5C74056F4E700375A300AEDA
:1002FE005BAF5C74066F4E700375A300AE5BAF5CB4
:10030E0074076F4E700375A300AE5BAF5C74086F1D
:10031E004E700375A300AE5BAF5C7408BE00039F06
:10032E005016AC59AD5AED2FFFEC3EFE9000681200
:10033E005F3CE5A3F075A300AE5BAF5CEFB41009B4
:10034E00EEB401057414125EF5AE5BAF5CEFB41043
:10035E0007EEB4010375F80D785B125F6902029126
:10036E0022755C00755B0075F809AE5BAF5C7417A7
:10037E00BE0004D39F5003020447A2F9B3500302F8
:10038E000444E55C455B700375A3D2AE5BAF5C7451
:10039E00016F4E700375A300AE5BAF5C74026F4EBF
:1003AE00700D9007B2E075F002A4FDACF08DA3AE17
:1003BE005BAF5C74036F4E700375A300AE5BAF5CF6
:1003CE0074046F4E700375A300AE5BAF5C74056F63
:1003DE004E700375A300AE5BAF5C74066F4E700378
:1003EE0075A300AE5BAF5C74076F4E700375A30010
:1003FE00AE5BAF5C74086F4E700375A300AE5BAF5F
:10040E005C7408BE00039F500C90004A125F3CE5DE
:10041E00A3F075A300AE5BAF5C74166F4E700574DF
:10042E0014125EF5AE5BAF5C74166F4E700375F80A
:10043E000D785B125F690203782290003DE0B4AB49
:10044E000280030204E2755C00755B0075F809AE6C
:10045E005BAF5C7412BE007CD39F4078A2F9B340B0
:10046E0070E55C455B700375A382AE5BAF5C740197
:10047E006F4E700375A300AE5BAF5C74026F4E706F
:10048E000D9007B2E075F002A4FDACF08DA3AE5B4B
:10049E00AF5C74036F4E700375A300AE5BAF5C74FC
:1004AE0003BE00039F500990004F125F3CE0F5A37E
:1004BE00AE5BAF5C74116F4E70057414125EF5AEC8
:1004CE005BAF5C74116F4E700375F80D785B125F45
:1004DE006902045D229007BCE4F074649007B1F8E1
:1004EE00E4F0E8A3F012036F74C89007B1F8E4F0DB
:1004FE00E8A3F0900056E0B4371A900053E0900055
:10050E004AF0900054E090004BF0900055E09000BF
:10051E004CF080469007BC7401F074659007B1F8FA
:10052E00E4F0E8A3F012036F74C89007B1F8E4F09A
:10053E00E8A3F0900056E0B4371A900053E0900014
:10054E004AF0900054E090004BF0900055E090007F
:10055E004CF0800674029007BCF09007BDE4F07476
:10056E00669007B1F8E4F0E8A3F012036F74C89038
:10057E0007B1F8E4F0E8A3F0900055E0B43712901C
:10058E000053E0900044F0900054E090004DF08055
:10059E00769007BD7401F074679007B1F8E4F0E847
:1005AE00A3F012036F74C89007B1F8E4F0E8A3F05B
:1005BE00900055E0B43712900053E0900044F09054
:1005CE000054E090004DF0803E74029007BDF07430
:1005DE00689007B1F8E4F0E8A3F012036F74C890C6
:1005EE0007B1F8E4F0E8A3F0900055E0B4371290AC
:1005FE000053E0900044F0900054E090004DF080E5
:10060E000674039007BDF022E54E64046006E5997A
:10061E0064FF6002802AA2374004D2378020E54E64
:10062E00600874E6254E900040F0754E00E54D6072
:10063E000874F0254D900040F0754D00C2378002D1
:10064E00C237E54E9033F8F8282873754E00E599B9
:10065E00B4FF03754D01E599B4FE03754D02E5999E
:10066E00B4FD03754D03E599B4FC03754D04E5998E
:10067E00B4FA03754D05E599B4FB06754E01123AB1
:10068E0082E599B4F906754E04123A82E599D3942F
:10069E00E54007E599C394F04002801685994F75A1
:1006AE004E027E017F00E54FC394E6125F158E3237
:1006BE008F339007B5E4F0A3F0E599D394C44007C7
:1006CE00E599C394E64002802885994F754E0374D0
:1006DE00E5C3954FF533753200AE32AF339057FD0B
:1006EE00125EE4E493F87401939007B5C8F0A3C8C2
:1006FE00F0D299020AB3900053E070429007B5E031
:10070E00FEA3E0FF74FFBE00039F5009EFC39446A3
:10071E00EE940640119007B5E0FEA3E0FFEFD394F0
:10072E006DEE940640139007B5E0FEA3E0FF900037
:10073E0071125F3CE599F0800385997380119007E3
:10074E00B5E0FEA3E0FF900071125F3CE599F090DA
:10075E0007B5125F239007B5E0FEA3E0FFEFB401EB
:10076E0006EEB40702800302089B900771E0B43CCA
:10077E00028003020885C29C900053E090010FF0A6
:10078E00900054E090007EF0900055E090009EF0B6
:10079E00900056E09000C7F0900057E0900073F084
:1007AE00900058E09000B9F0900059E09000D7F01A
:1007BE0090005AE09000ABF090005BE09000C9F022
:1007CE0090005CE09000F9F01236F0900065E09039
:1007DE0000E0F0900066E0900097F0900067E090E7
:1007EE000098F074639007B1F8E4F0E8A3F074ABEE
:1007FE0090003DF012044890003DE4F075096475D8
:10080E0008001200E3A21F4038757201E572D394FE
:10081E0007502CE5729007B1F8E4F0E8A3F074AA43
:10082E0090003DF012010FE572C39407500975094F
:10083E00647508001200E37872740126F650CD80BC
:10084E0036757208E572D3940E502CE5729007B18E
:10085E00F8E4F0E8A3F074AA90003DF012010FE561
:10086E0072C3940E50097509647508001200E3787E
:10087E0072740126F650CD74C89007B1F8E4F0E812
:10088E00A3F0D29C754E00754D007599FB020AB30C
:10089E009007B5E0FEA3E0FFEF4E70068599317527
:1008AE0030009007B5E0FEA3E0FF74016F4E701BA1
:1008BE00AC30AD31AA32AB33ED2BFBEC3AFA8A06F3
:1008CE008B07900071125F3CE599F09007B5125FAF
:1008DE00239007B5E0FEA3E0FF74026F4E7021ACCB
:1008EE0030AD3174566D4C7006E54F64E660028093
:1008FE0003123A821236F0854F99754E00754D00EF
:10090E00020AB39007B5E0FEA3E0FF900071125FFC
:10091E003CE599F09007B5125F239007B5E0FEA372
:10092E00E0FFAC32AD338F028E038C068D079058EC
:10093E003F125EE4E493F9740193FEEAD39EEB99C1
:10094E004009854F99754E00754D00020AB3900708
:10095E00B5E0FEA3E0FF900071125F3CE599F090C8
:10096E0007B5125F239007B5E0FEA3E0FFEFB400DA
:10097E0006EEB401028003020AB390004CE075F05B
:10098E0002A4FDACF08D72ED900071125F47EDFA8E
:10099E00E0FBEA900074125F47EBFAE0FBEA2BFAF9
:1009AE0090004CE0B502028003020AA50DED900006
:1009BE0071125F47E572FDE0FAED900075125F4728
:1009CE00EAFDE0FAEDC39AFD90004CE0B505028019
:1009DE0003020AA5E572900073125F47E572FDE00F
:1009EE00FAED900076125F47EAFDE0FAED2AFD90EF
:1009FE00004CE0B505028003020AA5E5729000776F
:100A0E00125F47FDE0FAED90004CE0F4042A9000EE
:100A1E0053F0E572900078125F47FDE0FAED90001A
:100A2E004CE0F4042A900054F0E572900079125FC5
:100A3E0047FDE0FAED90004CE0F4042A900055F0EA
:100A4E00E57290007A125F47FDE0FAED90004CE0FF
:100A5E00F4042A9007B1F8E4F0E8A3F074AB900028
:100A6E003DF01204487509647508001200E3900702
:100A7E00B1125F231204487509647508001200E371
:100A8E009007B1125F231204487599F975096475C0
:100A9E0008001200E380FE7599FF75096475080061
:050AAE001200E380FED0
:0F33F80002065902070402089E02091102095C2D
:100AB30022E54D903407F8282873020B989007B568
:100AC300E0FEA3E0FF900042125F3CE0F59990073F
:100AD300B5125F239007B5E0FEA3E0FF74116F4EDC
:100AE3007003754D00020B98856D99020B98900762
:100AF300B5E0FEA3E0FF900071125F3CE0F599EFD3
:100B0300B40107EEB40703754D009007B5125F23D8
:070B1300020B989007B6E009
:0F340700020ABD020AC0020AEB020AF1020B160A
:100B1A009035BAF82828738552998067855E99803E
:100B2A0062856099805D856499805885669980534D
:100B3A00856799804E85689980498569998044902E
:100B4A000016E0F599803CA238B340077599FAC2BD
:100B5A00388017A229B3400575990F800B90004081
:100B6A00E0F599900040E4F0C2298017856A9980DF
:100B7A0012856599800D856B9980087599FC8003AB
:030B8A00754D00A6
:1035BA00020B21020B26020B2B020B30020B3502E7
:1035CA000B3A020B3F020B44020B49020B51020B4E
:0D35DA0076020B7B020B80020B85020B8A30
:0B0B8D009007B5125F2380031235E7CC
:03341600020B9511
:100B980022E537255AFFAE5950010E900071125FB9
:100BA8003CE0F538E537255AFFAE5950010E0FBF26
:100BB80000010E900071125F3CE0F539853F3BE57E
:100BC80038B539058538378041E539D39538401D22
:100BD800E539C39538853AF0A4FFAEF0E53B8E04BD
:100BE8008F05FF125F05ED2538F537801DE538C301
:100BF8009539853AF0A4FFAEF0E53B8E048F05FFEA
:100C0800125F05EDF4042538F53722E539D3953818
:100C1800401DE539C39538853AF0A4FFAEF0E53BB1
:100C28008E048F05FF125F05ED2538F537801DE529
:100C380038C39539853AF0A4FFAEF0E53B8E048FB2
:100C480005FF125F05EDF4042538F537229000778B
:100C5800E0B40170E56675F00A84FF7E008F37E521
:100C68006675F00A84ADF07C008D3A753F0A7559B7
:100C780005755A24E537C394115005120B9980065F
:100C88009005A6E0F537E53790006AF0E56675F05F
:100C98000A84FF7E008F37E56675F00A84ADF07C24
:100CA800008D3A753F0A755905755A5AE537C39448
:100CB800115005120B9980069005DCE0F537E537F1
:100CC80090000EF022900077E0B4016AE56675F0B6
:100CD8000A84FF7E008F37E56675F00A84ADF07CE4
:100CE800008D3A753F0A755905755A36E537C3942C
:100CF800115005120B9980069005B8E0F537853735
:100D08004BE56675F00A84FF7E008F37E56675F05F
:100D18000A84ADF07C008D3A753F0A755905755AFD
:100D280048E537C394115005120B9980069005CAFF
:100D3800E0F53785374C22E55E75F00484FF7E00C8
:100D48008F37E55E75F00484ADF07C008D3A753F11
:100D580004755901755A00E537C3943F5005120BC5
:100D68009980069001B0E0F53785372975280090FD
:100D7800003FE075F020A4FFAEF09000C2E08E04C2
:100D88008F05FF125F058D379000AAE0D3955E505E
:100D980003020E459000CEE0D3955E4010ED900121
:100DA800B1125F47E0F52B752A00020E42900099B8
:100DB800E0D3955E4043E5379001B1125F47E0F517
:100DC80038E5379001D1125F47E0F5399000CEE061
:100DD800F404255EF53A900099E0FE9000CEE0F428
:100DE800042EF53BE538B539058538378003120CF4
:100DF8001385372B752A008041E5379001D1125FA2
:100E080047E0F538E5379001F1125F47E0F5399092
:100E18000099E0F404255EF53A9000AAE0FE9000FF
:100E280099E0F4042EF53BE538B539058538378067
:100E380003120C1385372B752A00020EEC9000D193
:100E4800E0D3955E5011E537900231125F47E0F527
:100E58002B752A00020EEC90009AE0D3955E504361
:100E6800E537900211125F47E0F538E53790023117
:100E7800125F47E0F53990009AE0F404255EF53AF0
:100E88009000D1E0FE90009AE0F4042EF53BE5389E
:100E9800B539058538378003120C1385372B752A29
:100EA800008041E5379001F1125F47E0F538E537FA
:100EB800900211125F47E0F5399000AAE0F404258A
:100EC8005EF53A90009AE0FE9000AAE0F4042EF550
:100ED8003BE538B539058538378003120C1385375B
:100EE8002B752A00229000E2E0F53C753F117559F8
:100EF80002755A00AE51AF52E53C75F00FA4FDAC37
:100F0800F0EDD39FEC9E4021E53C8E048F05FF1247
:100F18005F05ED75F010A4FFAEF0E55E75F0118485
:100F2800FD7C00ED2FF53D800EE55E75F01184FF28
:100F38007E00EF24F0F53D853D37E55E75F01184C0
:100F4800AFF07E008F3A120B9985373EAE51AF5203
:100F58009000E2E075F00FA4FDACF0EDD39FEC9E9D
:100F68004028755902755A10853D37120B99853EF0
:100F780038853739AE51AF52E53C8E048F05FF12E4
:100F88005F308D3A853C3B120C1385372975280054
:100F9800752B64752A00229000E2E0F53C753F113C
:100FA800755902755A00AE51AF52E53C75F00FA461
:100FB800FDACF0EDD39FEC9E4021E53C8E048F05FF
:100FC800FF125F05ED75F010A4FFAEF0E56075F057
:100FD8001184FD7C00ED2FF53D800EE56075F01164
:100FE80084FF7E00EF24F0F53D853D37E56075F020
:100FF8001184AFF07E008F3A120B9985373EAE51BF
:10100800AF529000E2E075F00FA4FDACF0EDD39F75
:10101800EC9E4028755902755A10853D37120B9978
:10102800853E38853739AE51AF52E53C8E048F0581
:10103800FF125F308D3A853C3B120C1385372975BA
:1010480028009000ACE0B40453E55E75F00484FF1A
:101058007E008F37E55E75F00484ADF07C008D3A34
:10106800753F04755901755A00E537C3943F50051B
:10107800120B9980069001B0E0F537AE28AF29E54C
:1010880037125F1574648E048F05FF125F05AE2852
:10109800AF29EF2DFDEE3CFC8C288D29752B64754E
:1010A8002A0022900077E0B40146E56675F00A84CC
:1010B800FF7E008F37E56675F00A84ADF07C008D01
:1010C8003A753F0A755905755A00E537C3941150AA
:1010D80005120B998006900582E0F537AE2AAF2BF2
:1010E800E5372FFF50010E7464125F598E2A8F2B3B
:1010F800900078E0B40146E56775F00A84FF7E0049
:101108008F37E56775F00A84ADF07C008D3A753F3E
:101118000A755905755A6CE537C394115005120BB9
:101128009980069005EEE0F537AE2AAF2BE5372F0C
:10113800FF50010E7464125F598E2A8F2B9000871E
:10114800E0B40249E569C3944175F00584FF7E0067
:101158008F37E56975F00584ADF07C008D3A753FF1
:1011680005755906755A00E537C394135005120BD7
:10117800998006900684E0F537AE2AAF2BE5372F25
:10118800FF50010E7464125F598E2A8F2B9000C98C
:10119800E0B40202800302124AE55E75F01584FF8E
:1011A8007E008F37E55E75F01584ADF07C008D3AD2
:1011B800753F15755903755AF4E537C3940B5005F7
:1011C800120B998006900470E0F537E53775F0FF4B
:1011D800A4FFAEF09000CAE08E048F05FF125F05F1
:1011E800ED900063F0E56575F078A4FFAEF074FF4C
:1011F8008E048F05FF125F058C598D5A74028C0678
:101208008D071200398F37AC59AD5A7404FF125F3D
:10121800308D3A753F04755906755A28E537C394D9
:101228001D5005120B9980069006B6E0F537AE2AD8
:10123800AF2BE5372FFF50010E7464125F598E2AC9
:101248008F2B900076E0B4025DE56075F064A4FF32
:10125800AEF074081200398E5B8F5C74058E048FB3
:1012680005FF125F058D37AE5BAF5C74058E048F8A
:1012780005FF125F308D3A753F05755905755ADEC1
:10128800E537C394135005120B998006900662E067
:10129800F537AE2AAF2BE5372FFF50010E746412D5
:1012A8005F598E2A8F2B9000B8E0703C90003FE089
:1012B80075F00584FF7E008F3790003FE075F005DC
:1012C80084ADF07C008D3A753F05755905755AC097
:1012D800E537C3941D5005120B99800690064EE021
:1012E800F537E53790006BF02290007FE0B40117E6
:1012F8009007B8E0252BFFAE2A50010E9000D3E0EE
:10130800125F598E2A8F2B9000F7E0B401149000D9
:10131800F8E0A851B8000495525007E55EC3955F00
:10132800400280129000A1E0252BFFAE2A50010E4A
:101338008E2A8F2B802F90007FE0B40316A22BB348
:10134800B350109007BBE0C39405A851B8000695A8
:1013580052400280109000A1E0252BFFAE2A5001D8
:101368000E8E2A8F2B900079E0B4020280030215BA
:101378004D90007CE0602FE566D3944640289000AD
:101388000FE0FEA3E0FF9000B7E075F003A4FDAC0A
:10139800F0EFD39DEE9C400E9000DBE0A851B80022
:1013A80005D39552500302154D9000C4E0855EF0B8
:1013B800A4FFAEF07405125F1574071200398E5938
:1013C8008F5A900083E0A851B800049552501290AB
:1013D8000084E075F002A4FDACF0EFC39DEE9C40E4
:1013E8000302154DE55E75F00B84FF7E0090060143
:1013F800125F3CFEE0FFEE90007BE0FEEF8E00887F
:10140800F0A4FFAEF074648E048F05FF125F058CA4
:10141800598D5A90003FE075F018A4FFAEF0900087
:10142800C2E08E048F05FF125F058C068D079006BB
:1014380019125F3CAE59AF5AE0125F1574648E04FE
:101448008F05FF125F058C598D5AE564A859B800BD
:1014580077D3955A4072E564C3955AFFE49559FECF
:101468008E598F5A7428BE00039F500C755A2875E0
:101478005900740D900040F0AE59AF5A90007CE0CE
:10148800125F1574288E048F05FF125F058C598D25
:101498005AAE28AF29740A8E048F05FF125F058D96
:1014A800068C07AC59AD5ACFCECF120003740A8E02
:1014B800048F05FF125F058C598D5AAE28AF29128B
:1014C8005F618E288F29807DE564A859B80004954E
:1014D8005A5072AE59AF5AE564125F598E598F5AF5
:1014E8007428BE00039F500C755A28755900740D56
:1014F800900040F0AE59AF5A90007CE0125F15742E
:10150800288E048F05FF125F058C598D5AAE28AFBF
:1015180029740A8E048F05FF125F058D068C07ACAF
:1015280059AD5ACFCECF120003740A8E048F05FF2F
:10153800125F058C598D5AAE28AF29EF2DFDEE3C70
:10154800FC8C288D29229000D7E0B4026AE55E75EC
:10155800F00884FF7E008F37E55E75F00884ADF0F3
:101568007C008D3A753F08755901755AE0E537C317
:10157800943F5005120B998006900270E0F537856C
:10158800372D752C00AE2CAF2DAC2AAD2B120003D5
:1015980074648E048F05FF125F058C2C8D2D9000CE
:1015A80074E08C068D07125F1574648E048F05FF36
:1015B800125F058C2C8D2DAE28AF29AC2AAD2B12CD
:1015C800000374648E048F05FF125F058C288D2933
:1015D800900074E08C068D07125F1574648E048F7A
:1015E80005FF125F058C288D29A20D401DAE51AF55
:1015F800527405BE00039F5002D20DE560D394CC0F
:101608004008D2017411900040F09000D6E0B40276
:10161800089000D8E0640160028035AE28AF29E563
:101628006A125F1574E78E048F05FF125F058C2818
:101638008D299000D7E0B40217AE2CAF2DE56A12C1
:101648005F1574E78E048F05FF125F058C2C8D2DB6
:10165800900096E05402601B90008DE0A851B800FD
:1016680012D39552400DA20DB3B35007E560C39451
:101678009A40028028AE35AF3690008BE075F002B4
:10168800A4FDACF0EF2DFDEE3CFC74022DFD5001E5
:101698000CE560BC0007D39D4003754301856036A7
:1016A800753500E54370030217919000E9E0C39592
:1016B8004350030217839000F9E0C394025076E583
:1016C8006675F00A84FF7E00900571125F3CE0F5B4
:1016D8005A755900AE59AF5A90008CE0125F1574D4
:1016E800648E048F05FF125F058C5B8D5C9000E9AA
:1016F800E004C395438C068D07125F159000E9E05E
:101708008E048F05FF125F058C5B8D5CAE28AF29B8
:10171800EF2DFDEE3CFC8C288D299000D7E0B4021B
:1017280012AE2CAF2DAA5BAB5CEF2BFBEE3AFA8A1C
:101738002C8B2D80469000E9E004C39543854BF03F
:10174800A4FFAEF09000E9E08E048F05FF125F055C
:101758008C5B8D5CAE28AF29EF2DFDEE3CFC8C2810
:101768008D299000D7E0B40212AE2CAF2DAA5BAB46
:101778005CEF2BFBEE3AFA8A2C8B2D05439000E99F
:10178800E0C395435003754300900096E054016010
:101798001B90008AE0A851B80012D39552400DA2C0
:1017A8000DB3B35007E55EC394CC4002802590008A
:1017B80088E075F003A4FFAEF0E5402FFF50010E5E
:1017C80074032FFF50010EE55EBE0007D39F400350
:1017D800754401855E40E54470030218C49000EA30
:1017E800E0C3954450030218B69000F9E0C3940290
:1017F8005076E56675F00A84FF7E00900571125FE9
:101808003CE0F55A755900AE59AF5A900089E0127C
:101818005F1574648E048F05FF125F058C5B8D5C09
:101828009000EAE004C395448C068D07125F15907A
:1018380000EAE08E048F05FF125F058C5B8D5CAEBD
:1018480028AF29EF2DFDEE3CFC8C288D299000D780
:10185800E0B40212AE2CAF2DAA5BAB5CEF2BFBEE13
:101868003AFA8A2C8B2D80469000EAE004C395440E
:10187800854CF0A4FFAEF09000EAE08E048F05FFDF
:10188800125F058C5B8D5CAE28AF29EF2DFDEE3C19
:10189800FC8C288D299000D7E0B40212AE2CAF2D15
:1018A800AA5BAB5CEF2BFBEE3AFA8A2C8B2D054436
:1018B8009000EAE0C3954450037544009000ECE0C2
:1018C8002529FFAE2850010E8E288F2990009BE015
:1018D800A828B800049529500990009BE0F52975BF
:1018E80028009000D7E0B4020D90009BE0A82CB827
:1018F8000006952D4002800990009BE0F52D752C7F
:1019080000229000D7E0B401028003021A15A20D4C
:10191800B35003021A139000A2E0B40168AE28AFD6
:1019280029AC51AD52120003743C8E048F05FF128E
:101938005F059000B2E0BC00109D400D9000B4E03F
:10194800A828B8000495295002D202AE28AF29ACC5
:1019580051AD52120003743C8E048F05FF125F05CF
:101968009000B2E0C3940ABC0015D39D40119000CA
:10197800B4E0C39405A828B80005D395295002807F
:1019880002C2028068AE28AF29AC51AD52120003E2
:1019980074788E048F05FF125F059000B2E0BC00DA
:1019A800109D400D9000B4E0A828B8000495295077
:1019B80004D2028038AE28AF29AC51AD52120003D0
:1019C80074788E048F05FF125F059000B2E0C3940F
:1019D8000ABC0015D39D40119000B4E0C39405A83B
:1019E80028B80005D3952950028002C202A202B38A
:1019F8004019AE28AF299000B3E0125F1574648EC9
:101A0800048F05FF125F058C288D298002C202A26F
:101A180000B34006A201B3B35009900015E4F0A347
:101A2800F08024AE28AF297400D39F74019E400C27
:101A3800900015E528F0A3E529F0800B74FF9000CD
:101A480015F8E4F0E8A3F09000B9E0D39402400C54
:101A58009000A4E07006A20DB3B34002801AAE282D
:101A6800AF297402125F158E288F29AE2CAF2D7402
:101A780002125F158E2C8F2D9000A2E0B4011AAED1
:101A880028AF297402125F158E288F29AE2CAF2D2E
:101A98007402125F158E2C8F2DAE28AF29745E123A
:101AA8005F15740A8E048F05FF125F058C288D2937
:101AB8009000D7E0B40217AE2CAF2D745E125F15FC
:101AC800740A8E048F05FF125F058C2C8D2DAE28AD
:101AD800AF297402BE000AD39F40067529027528F3
:101AE80000AE2CAF2D7402BE000AD39F4006752DA0
:101AF80002752C00900013E528F0A3E529F0229048
:101B0800003FE0900371125F47E0F5417542649031
:101B1800003FE0FE9000ADE0D39E4037E55E75F0F3
:101B28000884FF7E008F37E55E75F00884ADF07C91
:101B3800008D3A753F08755903755A96E537C39471
:101B48001F5005120B998006900426E0F53785375B
:101B5800428035E55E75F00884FF7E008F37E55ECC
:101B680075F00884ADF07C008D3A753F087559030F
:101B7800755AB6E537C3941F5005120B9980069025
:101B88000446E0F537853742229000E3E0F53C75DE
:101B98003F11755904755A00AE51AF52E53C75F0C6
:101BA8000FA4FDACF0EDD39FEC9E4021E53C8E04E4
:101BB8008F05FF125F05ED75F010A4FFAEF0E55E2E
:101BC80075F01184FD7C00ED2FF53D800EE55E7506
:101BD800F01184FF7E00EF24F0F53D853D37E55E8A
:101BE80075F01184AFF07E008F3A120B9985373E5D
:101BF800AE51AF529000E3E075F00FA4FDACF0EDEC
:101C0800D39FEC9E4028755904755A10853D3712AC
:101C18000B99853E38853739AE51AF52E53C8E0475
:101C28008F05FF125F308D3A853C3B120C138537C8
:101C380041754264229000E3E0F53C753F11755907
:101C480004755A00AE51AF52E53C75F00FA4FDACD7
:101C5800F0EDD39FEC9E4021E53C8E048F05FF12EA
:101C68005F05ED75F010A4FFAEF0E56075F0118426
:101C7800FD7C00ED2FF53D800EE56075F01184FFC9
:101C88007E00EF24F0F53D853D37E56075F0118461
:101C9800AFF07E008F3A120B9985373EAE51AF52A6
:101CA8009000E3E075F00FA4FDACF0EDD39FEC9E3F
:101CB8004028755904755A10853D37120B99853E91
:101CC80038853739AE51AF52E53C8E048F05FF1287
:101CD8005F308D3A853C3B120C1385374175426461
:101CE8009000DEE0B4047990003FE0FE9000ADE0A3
:101CF800D39E4037E55E75F00884FF7E008F37E598
:101D08005E75F00884ADF07C008D3A753F08755912
:101D180003755A96E537C3941F5005120B99800630
:101D2800900426E0F5378537428035E55E75F00882
:101D380084FF7E008F37E55E75F00884ADF07C0087
:101D48008D3A753F08755903755AB6E537C3941F20
:101D58005005120B998006900446E0F53785374206
:101D680022900077E0B4013BE56675F00A84FF7EB7
:101D7800008F37E56675F00A84ADF07C008D3A7502
:101D88003F0A755905755A12E537C3941150051263
:101D98000B998006900594E0F537E5422537C39402
:101DA80064F542900078E0B4013BE56775F00A8479
:101DB800FF7E008F37E56775F00A84ADF07C008DF3
:101DC8003A753F0A755905755A7EE537C39411501F
:101DD80005120B998006900600E0F537E542253795
:101DE800C39464F542E5412542F53490007FE0B4A0
:101DF80002109007B7E02534FE9000D3E0F4042EDB
:101E0800F5349000D6E0D394014040E56AC394E7E6
:101E1800501D74E7C3956AFE9007B9E08E00F5F08F
:101E2800E884FF7E008F37E5342537F534801CE5DC
:101E38006AC394E7FE9007B9E08E00F5F0E884FFE6
:101E48007E008F37E534C39537F534A20D4006E59B
:101E5800412464F534E534D394644009E534C394EB
:101E680064F53480037534009000AFE0C3953450B6
:101E7800069000AFE0F53422D200900069E0A85146
:101E8800B8000495525041900069E0A851B8000488
:101E98009552500375340F900069E004A851B800BA
:101EA800049552500375340A900069E02402A85141
:101EB800B8000495525005753405C200900069E0D9
:101EC80060067409900040F0C23B7E017F009000DC
:101ED800B5E0125F159000C4E08E048F05FF125F15
:101EE80005E55EBC0017D39D40139000BEE0B40228
:101EF80004D23B8002C200740A900040F09000B601
:101F0800E0C3956650159000C8E0A851B800049544
:101F1800525002C200740B900040F0E566C394640E
:101F2800501D90010EE0600D90010EE0A851B80020
:101F380006955240028008C200740B900040F0A23F
:101F48000040037534059000F7E0B401149000F8E0
:101F5800E0A851B8000495525007E55EC3955F406C
:101F68000280089000A0E0F534803A90007FE0B449
:101F78000306A22BB3B34002802B9007BBE0C394A7
:101F880005A851B800049552500C9000A0E0F53413
:101F9800740C900040F09007BBE0A851B80004957D
:101FA800525002C20085346B900071E02534FE90D7
:101FB800003FE075F01E84FC7F00EE2CF534229083
:101FC800003FE075F00584FF7E008F3790003FE00A
:101FD80075F00584ADF07C008D3A753F05755903A1
:101FE800755AD69000C2E01475F00584FF7E00E5AE
:101FF80037BE00039F5005120B99800BE5379004FC
:1020080047125F47E0F537E5379007BAF09007BA0F
:10201800E0FE9000B1E0C39E50089000B1E0900748
:10202800BAF022E56675F00A84FF7E009005711209
:102038005F3CE0F546E546D394644010E546C3941A
:102048006475F00F84FF7E008F468003754600900C
:102058000094E02546F546229007ABE0FEA3E0FF9A
:102068007404120039E55E125F15740F8E048F0533
:10207800FF125F059007A9ECF0A3EDF0900087E050
:10208800B40262E569C3944175F00584FF7E008F50
:1020980037E56975F00584ADF07C008D3A753F052C
:1020A800755906755A14E537C394175005120B99DC
:1020B8008006900698E0F5379007A9E0FEA3E0FFB8
:1020C800740A8E048F05FF125F05E5378C068D07AD
:1020D800125F15740A8E048F05FF125F059007A919
:1020E800ECF0A3EDF09007A9E0FEA3E0FF9007AFA6
:1020F800E0FCA3E0FDEDD39FEC9E400F9007AFE01E
:10210800F8A3E09007A9C8F0A3C8F0229006B8E0A9
:10211800903419F8282873804C85527280479000B3
:10212800C4E0855EF0A4FFAEF074081200398F7227
:102138008033856072802E856672802985677280FB
:1021480024856872801F856972801A856A72801575
:102158008565728010856472800B856B728006902D
:052168000016E0F57215
:1034190002211F02212102212602213A02213F0213
:10342900214402214902214E02215302215802213D
:073439005D02216202216720
:10216D009006B9E0FE9006BAE0D39E404B9006B8BB
:10217D00E0B404189006BAE0C395725002D22C90C8
:10218D0006B9E0D395724002C22C802A9006B9E0C0
:10219D00C3957250099006BAE0D395725002800231
:1021AD00D22C9006B9E0D3957250099006BAE0C3CF
:1021BD0095725002C22C802A9006B9E0D3957240D8
:1021CD00099006BAE0C3957240028002C22C9006B7
:1021DD00B9E0C3957240099006BAE0D395724002FA
:1021ED00D22C229006BCE0903440F8282873804C05
:1021FD0085527280479000C4E0855EF0A4FFAEF07A
:10220D0074081200398F728033856072802E856656
:10221D007280298567728024856872801F85697236
:10222D00801A856A7280158565728010856472804A
:0C223D000B856B728006900016E0F572B5
:103440000221FB0221FD02220202221602221B029D
:10345000222002222502222A02222F0222340222C4
:073460003902223E02224363
:102249009006BDE0FE9006BEE0D39E405F9006BCBE
:10225900E0B404189006BEE0C395725002D22D90E6
:1022690006BDE0D395724002C22D803E9006BDE0C6
:10227900C3957250099006BEE0D395725002800250
:10228900D22D9006BDE0D3957250099006BEE0C3E9
:1022990095725002C22D9006BCE0B401099000D09D
:1022A900E0D3956050028002C22D802A9006BDE0DD
:1022B900D3957240099006BEE0C395724002800230
:1022C900C22D9006BDE0C3957240099006BEE0D3C9
:1022D90095724002D22D229006C0E0903467F8280A
:1022E9002873804C85527280479000C4E0855EF067
:1022F900A4FFAEF074081200398F728033856072C2
:10230900802E85667280298567728024856872802F
:102319001F856972801A856A7280158565728010B9
:10232900856472800B856B728006900016E0F572E9
:103467000222EB0222ED0222F202230602230B02C2
:10347700231002231502231A02231F0223240223E7
:073487002902232E0223336A
:102339009006C1E0FE9006C2E0D39E404B9006C0D5
:10234900E0B404189006C2E0C395725002D22E90F0
:1023590006C1E0D395724002C22E802A9006C1E0E0
:10236900C3957250099006C2E0D39572500280025B
:10237900D22E9006C1E0D3957250099006C2E0C3EF
:1023890095725002C22E802A9006C1E0D395724000
:10239900099006C2E0C3957240028002C22E9006DF
:1023A900C1E0C3957240099006C2E0D3957240021C
:1023B900D22E229006C4E090348EF8282873804CDF
:1023C90085527280479000C4E0855EF0A4FFAEF0AC
:1023D90074081200398F728033856072802E856689
:1023E9007280298567728024856872801F85697269
:1023F900801A856A7280158565728010856472807D
:0C2409000B856B728006900016E0F572E7
:10348E000223C70223C90223CE0223E20223E7024C
:10349E0023EC0223F10223F60223FB022400022472
:0734AE000502240A02240FAD
:102415009006C5E0FE9006C6E0D39E404B9006C4EC
:10242500E0B404189006C6E0C395725002D22F900E
:1024350006C5E0D395724002C22F802A9006C5E0FA
:10244500C3957250099006C6E0D39572500280027A
:10245500D22F9006C5E0D3957250099006C6E0C309
:1024650095725002C22F802A9006C5E0D39572401E
:10247500099006C6E0C3957240028002C22F9006FD
:10248500C5E0C3957240099006C6E0D39572400237
:10249500D22F229006C8E09034B5F8282873804CD6
:1024A50085527280479000C4E0855EF0A4FFAEF0CF
:1024B50074081200398F728033856072802E8566AC
:1024C5007280298567728024856872801F8569728C
:1024D500801A856A728015856572801085647280A0
:0C24E5000B856B728006900016E0F5720B
:1034B5000224A30224A50224AA0224BE0224C302D4
:1034C50024C80224CD0224D20224D70224DC0224FB
:0734D500E10224E60224EBF2
:1024F1009006C9E0FE9006CAE0D39E404B9006C804
:10250100E0B404189006CAE0C395725002D230902C
:1025110006C9E0D395724002C230802A9006C9E014
:10252100C3957250099006CAE0D395725002800299
:10253100D2309006C9E0D3957250099006CAE0C323
:1025410095725002C230802A9006C9E0D39572403C
:10255100099006CAE0C3957240028002C23090061B
:10256100C9E0C3957240099006CAE0D39572400252
:10257100D230229006CCE09034DCF8282873804CCD
:1025810085527280479000C4E0855EF0A4FFAEF0F2
:1025910074081200398F728033856072802E8566CF
:1025A1007280298567728024856872801F856972AF
:1025B100801A856A728015856572801085647280C3
:0C25C1000B856B728006900016E0F5722E
:1034DC0002257F02258102258602259A02259F025C
:1034EC0025A40225A90225AE0225B30225B8022582
:0734FC00BD0225C20225C735
:1025CD009006CDE0FE9006CEE0D39E404B9006CC1B
:1025DD00E0B404189006CEE0C395725002D231904B
:1025ED0006CDE0D395724002C231802A9006CDE02F
:1025FD00C3957250099006CEE0D3957250028002B9
:10260D00D2319006CDE0D3957250099006CEE0C33D
:10261D0095725002C231802A9006CDE0D39572405A
:10262D00099006CEE0C3957240028002C231900639
:10263D00CDE0C3957240099006CEE0D3957240026D
:10264D00D231229006D0E0903503F8282873804CC3
:10265D0085527280479000C4E0855EF0A4FFAEF015
:10266D0074081200398F728033856072802E8566F2
:10267D007280298567728024856872801F856972D2
:10268D00801A856A728015856572801085647280E6
:0C269D000B856B728006900016E0F57251
:1035030002265B02265D02266202267602267B02E3
:10351300268002268502268A02268F022694022608
:073523009902269E0226A377
:1026A9009006D1E0FE9006D2E0D39E404B9006D032
:1026B900E0B404189006D2E0C395725002D2329069
:1026C90006D1E0D395724002C232802A9006D1E049
:1026D900C3957250099006D2E0D3957250028002D8
:1026E900D2329006D1E0D3957250099006D2E0C358
:1026F90095725002C232802A9006D1E0D395724079
:10270900099006D2E0C3957240028002C232900657
:10271900D1E0C3957240099006D2E0D39572400288
:10272900D232229006D4E090352AF8282873804CBA
:1027390085527280479000C4E0855EF0A4FFAEF038
:1027490074081200398F728033856072802E856615
:102759007280298567728024856872801F856972F5
:10276900801A856A72801585657280108564728009
:0C2779000B856B728006900016E0F57274
:10352A0002273702273902273E022752022757026B
:10353A00275C02276102276602276B02277002278F
:07354A007502277A02277FBA
:102785009006D5E0FE9006D6E0D39E404B9006D449
:10279500E0B404189006D6E0C395725002D2339087
:1027A50006D5E0D395724002C233802A9006D5E063
:1027B500C3957250099006D6E0D3957250028002F7
:1027C500D2339006D5E0D3957250099006D6E0C372
:1027D50095725002C233802A9006D5E0D395724097
:1027E500099006D6E0C3957240028002C233900676
:1027F500D5E0C3957240099006D6E0D395724002A4
:10280500D233229006D8E0903551F8282873804CB1
:1028150085527280479000C4E0855EF0A4FFAEF05B
:1028250074081200398F728033856072802E856638
:102835007280298567728024856872801F85697218
:10284500801A856A7280158565728010856472802C
:0C2855000B856B728006900016E0F57297
:1035510002281302281502281A02282E02283302F3
:10356100283802283D02284202284702284C022816
:073571005102285602285BFD
:102861009006D9E0FE9006DAE0D39E404B9006D860
:10287100E0B404189006DAE0C395725002D23490A5
:1028810006D9E0D395724002C234802A9006D9E07D
:10289100C3957250099006DAE0D395725002800216
:1028A100D2349006D9E0D3957250099006DAE0C38C
:1028B10095725002C234802A9006D9E0D3957240B5
:1028C100099006DAE0C3957240028002C234900694
:1028D100D9E0C3957240099006DAE0D395724002BF
:1028E100D234229006DCE0903578F8282873804CA9
:1028F10085527280479000C4E0855EF0A4FFAEF07F
:1029010074081200398F728033856072802E85665B
:102911007280298567728024856872801F8569723B
:10292100801A856A7280158565728010856472804F
:0C2931000B856B728006900016E0F572BA
:103578000228EF0228F10228F602290A02290F027E
:10358800291402291902291E02292302292802299D
:073598002D02293202293740
:10293D009006DDE0FE9006DEE0D39E404B9006DC77
:10294D00E0B404189006DEE0C395725002D23590C3
:10295D0006DDE0D395724002C235802A9006DDE097
:10296D00C3957250099006DEE0D395725002800235
:10297D00D2359006DDE0D3957250099006DEE0C3A6
:10298D0095725002C235802A9006DDE0D3957240D3
:10299D00099006DEE0C3957240028002C2359006B2
:1029AD00DDE0C3957240099006DEE0D395724002DA
:1029BD00D23522AE2EAF2F74F5D39F74019E4008F1
:1029CD00782E125F69022ADA752F01752E00AE512D
:1029DD00AF52E546BE000DD39F40099000A6E0D34F
:1029ED00954740028023754700E546C39552F57221
:1029FD009000A9E0D395454008E5452572F5458041
:102A0D00069000A9E0F54580020547900082E0D3CD
:102A1D009560401CE55EC3955F4015AE51AF52E524
:102A2D0046BE00039F50099000A7E0D39548400291
:102A3D00806E9007BEE0A851B80004955250037502
:102A4D004A009007BEE0A851B8000BD3955240063E
:102A5D00E5529007BEF0E54A7041E552C39546F543
:102A6D0072E572D3940540037572059000A8E0C31A
:102A7D0095455007E572C3954540028009E545C36C
:102A8D009572F54580069000A8E0F5459000A8E008
:102A9D00D3954540069000A8E0F5457548008002A5
:102AAD000548E54A7016900082E0C39560500DE52B
:102ABD00462405A851B8000695524002800F90009B
:102ACD0095E0F545754A0174789007BEF022AE2E5B
:102ADD00AF2F74E9D39F74039E4008782E125F695F
:102AED00022C79752F01752E00754532A236402ABC
:102AFD00754519900095E075F002A4FFAEF0E5471D
:102B0D00BE0006D39F4002D2360547754A0374783E
:102B1D009007BEF0754900022C68AE51AF52E546E4
:102B2D006F4E7003022C68E546BE000DD39F400921
:102B3D009000A6E0D395474002800F754700E54A07
:102B4D00C394035003754519800DE546C39552F5A1
:102B5D0072E5472572F547900082E0D39560400EEF
:102B6D009007BEE0A851B80007D395524002800CE3
:102B7D000549900095E0B54903754A00E54AB4034F
:102B8D0006A20DB3B34002800A0549E549B43C03E2
:102B9D00754A02E54AB402299007BEE0A851B80073
:102BAD000ED395524009E5529007BEF0754900903D
:102BBD000082E0C39560500975490074789007BE96
:102BCD00F0E54A705A900082E0D39560401CE55EB6
:102BDD00C3955F4015AE51AF52E546BE00039F5001
:102BED00099000A7E0D3954840028008754800750C
:102BFD00454B8028E552C39546F572E572D3940591
:102C0D004003757205900082E0D395604008E54859
:102C1D002572F5488006E5482406F548754900E516
:102C2D004A7016900082E0C39560500DE54624056C
:102C3D00A851B80006955240028003754A01E54A35
:102C4D00B401187545190549900095E0B54906750B
:102C5D004A0275490074789007BEF0E54575F00A93
:102C6D00A4FFAEF09007B3EEF0A3EFF022E56E9067
:102C7D00359FF828287390007AE07003022E289073
:102C8D0000B0E0B401028003022D7890003EE0B563
:102C9D005D028003022D757E017F00E5BE125F157A
:102CAD00E5BD2FFF50010E8E598F5A7410125F150E
:102CBD00900068E08E048F05FF125F059007BFEC52
:102CCD00F0A3EDF0E56A60089000D6E064026002C2
:102CDD0080269000D8E0B4011F9007BFE0FEA3E06E
:102CED00FF74E7125F15E56A8E048F05FF125F050D
:102CFD009007BFECF0A3EDF090007AE0B4022790BE
:102D0D0007C1E0FEA3E0FF9007BFE0FCA3E0FDEFED
:102D1D002DFDEE3CFC74018C068D071200399007D9
:102D2D00BFEEF0A3EFF09007BFE0FEA3E0FF90072A
:102D3D00C1E0FCA3E0FDEDD39FEC9E4004D23980B1
:102D4D0002B2399007BFE0F8A3E09007C1C8F0A325
:102D5D00C8F09000ACE064016006A239B3B3400244
:102D6D0080069007C0E0F55E022E26D2397E017FE7
:102D7D0000E5BE125F15E5BD2FFF50010E8E598F78
:102D8D005A7410125F15900068E08E048F05FF12C3
:102D9D005F059007BFECF0A3EDF0E56A60089000C9
:102DAD00D6E06402600280269000D8E0B4011F9046
:102DBD0007BFE0FEA3E0FF74E7125F15E56A8E041E
:102DCD008F05FF125F059007BFECF0A3EDF09000AB
:102DDD007AE0B402279007C1E0FEA3E0FF9007BFA1
:102DED00E0FCA3E0FDEF2DFDEE3CFC74018C068DA7
:102DFD00071200399007BFEEF0A3EFF09007BFE088
:102E0D00F8A3E09007C1C8F0A3C8F09000ACE0644F
:102E1D000160069007C0E0F55E8003755E009000CE
:102E2D0076E07006756E01022C7A75BB180233F3CD
:102E3D00900076E07003022FC97E017F00E5BE127F
:102E4D005F15E5BD2FFF50010E8E598F5A9000BCB6
:102E5D00E0B4010F7E0F7FFFAC59AD5A125F618E4A
:102E6D00598F5A9000E1E0B40245AE59AF5A900027
:102E7D001FE0FCA3E0FDEDD39FEC9E400A90001FE8
:102E8D00E559F0A3E55AF0AE59AF5A900021E0FC98
:102E9D00A3E0FDEFD39DEE9C400A900021E559F093
:102EAD00A3E55AF0AE59AF5A74041200398F6090F1
:102EBD0000E1E0704CAE59AF5A90001FE0FCA3E06A
:102ECD00FDEFD39DEE9C4009125F618E598F5A80A4
:102EDD0006755A00755900AE59AF5A7410125F1528
:102EED00900065E08E048F05FF125F058C598D5A99
:102EFD0074FFBC0009D39D4005855A608003756041
:102F0D00FE9000ACE0B401028003022FC7A20DB306
:102F1D00B3500E900080E0A851B80005D3955250E3
:102F2D0003022FBC900081E075F019A4FFAEF09064
:102F3D0000C4E08E048F05FF125F059000BDE08593
:102F4D0060F0A4FFAEF074648D028C038E048F05C7
:102F5D00FF125F05EA2DFDEB3CFC8C598D5AE56A9D
:102F6D00600F9000D6E0B402089000D8E0640160D4
:102F7D00028017AE59AF5A74E7125F15E56A8E04D9
:102F8D008F05FF125F058C598D5AAE59AF5A9007B8
:102F9D00BFE0FCA3E0FDEDD39FEC9E4005855A5E9E
:102FAD00800BA239B340069007C0E0F55E800BA2FE
:102FBD0039B340069007C0E0F55E80037560009060
:102FCD000079E07006756E02022C7A75BB1902331A
:102FDD00F3900079E0700302307EE55DD3955040AB
:102FED000302307C90001DE0FEA3E0FFE564125F5C
:102FFD005990001DEEF0A3EFF07E017F00E5BE12AB
:10300D005F15E5BD2FFF50010E8E598F5A9000E6CA
:10301D00E07013740A125F1574518E048F05FF1240
:10302D005F058D648019AE59AF5A740A125F158F02
:10303D00048E057E017F95CDCCCD125E038F64E5A8
:10304D0064D39464400375646490001DE0FEA3E0B6
:10305D00FFE5642FFF50010E90001DEEF0A3EFF081
:10306D0090007DE0048E048F05FF125F058D648056
:10307D00037564329000C9E07006756E03022C7AF8
:10308D0075BB130233F39000C9E0604A7E017F00E7
:10309D00E5BE125F15E5BD2FFF50010E8E598F5AFB
:1030AD0074041200398F659000CBE08565F0A4FDA6
:1030BD00ACF07464FF125F058D659000CAE0856504
:1030CD00F0A4FFAEF074FF8E048F05FF125F05EDC7
:1030DD00900064F08003756500900077E0700675D0
:1030ED006E04022C7A75BB170233F3900077E0B4AF
:1030FD000102800302318C7E017F00E5BE125F1557
:10310D00E5BD2FFF50010E8E598F5A9007C3E06019
:10311D00199007C3E01490588112008CE493FC744D
:10312D000193FDEDC39FEC9E400280069007C3E026
:10313D0014F09007C3E0C394B3501DAE59AF5A902D
:10314D0007C3E00490588112008CE493FC74019342
:10315D00FDEFC39DEE9C400280069007C3E004F096
:10316D009007C3E0FE90009DE08E0088F0A4FFAEB6
:10317D00F074648E048F05FF125F058D66800375F4
:10318D006600900078E07006756E05022C7A75BBAE
:10319D00160233F3900078E0B40102800302323559
:1031AD007E017F00E5BE125F15E5BD2FFF50010EBC
:1031BD008E598F5A9007C4E060199007C4E014909F
:1031CD0059EB12008CE493FC740193FDEDC39FEC5D
:1031DD009E400280069007C4E014F09007C4E0C33F
:1031ED0094B3501DAE59AF5A9007C4E0049059EBFB
:1031FD0012008CE493FC740193FDEFC39DEE9C4093
:10320D000280069007C4E004F09007C4E0FE900031
:10321D00A3E08E0088F0A4FFAEF074648E048F05D9
:10322D00FF125F058D67800375670075BB1F023345
:10323D00F37E017F00E5BE125F15E5BD2FFF500146
:10324D000E8E598F5A7409125F1574E68E048F0510
:10325D00FF125F058D6990007FE07006756E0702A5
:10326D002C7A75BB150233F390007FE070030233A7
:10327D008F7E017F00E5BE125F15E5BD2FFF50016A
:10328D000E8E598F5A74041200398F6890007FE0AA
:10329D00B401159000D3E08568F0A4FFAEF074077B
:1032AD00120039EF9007B8F090007FE0B40215904E
:1032BD0000D3E08568F0A4FFAEF07407120039EF7B
:1032CD009007B7F090007FE0B40302800302338DC6
:1032DD009000C0E070389000D3E0601CE568C394A6
:1032ED00195002D22BE568D394644002C22B900092
:1032FD009FE09007BBF08014E568C394195002D28B
:10330D003AE568D394324002C23AC22B80639000F2
:10331D009FE070349000D3E08568F0A4FFAEF074A8
:10332D00FF8E048F05FF125F05ED9007BBF0AE51C8
:10333D00AF52741EBE0006D39F4002D22BE560D360
:10334D0094E54002C22B8029E568C3940A500DAE66
:10335D0051AF52741EBE0004D39F50028002D22B77
:10336D00E560D394E54002C22B90009FE09007BB2F
:10337D00F09007BBE0C39405500674059007BBF0B1
:10338D0080037568009000D6E07006756E08022CFB
:10339D007A75BB1480509000D6E060397E017F00B5
:1033AD00E5BE125F15E5BD2FFF50010E8E598F5AE8
:1033BD00EFD39421EE940E4005756AFF8015AE593A
:1033CD00AF5A7410125F1574E38E048F05FF125FF0
:1033DD00058D6A8003756A0090007AE0600575BB03
:0633ED001A800375BB18F5
:10359F00022C83022E3D022FDE0230930230F802FE
:0B35AF0031A102323E0232750233A34C
:0533F300056ED2EC2282
:095F47002582F582500205832237
:0F008C0025E050020583258250020583F582226C
:105EE400EF2F500205832582F582E5833E2EF5834C
:015EF400228B
:105F5900CFC39FFF50011E22C3EF9DFFEE9CFE227F
:085F69000806B600021806222A
:0D5F2300A3E004F07006120049E004F02233
:0E003900048007C3CE13CECF13CFD5E0F6223E
:105E0300BC000FBE0008ED8FF084FFADF022E4FE6E
:105E1300FF22BE000DEF60FE54F0606F20E7030227
:105E23005EB9EAC0E0EBC0E078017A0075F001EEFC
:105E330020E710EF25E0FFEE33FE0AC5F023C5F09F
:105E430030E7F0EA5407F9096A7A007B0060010839
:105E5300C3EC9E40167004ED9F4010ED9FFDEC9E39
:105E6300FCE5F0CA4ACA03F5F08005E5F003F5F056
:105E7300C3EE13FEEF13FFD9D77908CACBCAD8D024
:105E8300EAFEEBFFD0E0FBD0E0FA22EC8FF084FCDB
:105E9300ED54F045F0C48FF084FEEDC454F045F0AA
:105EA300C48FF084FDEEC4FE54F02DFFEE540F3C7E
:105EB300FEADF07C0022790078008FF0EC7E0820A4
:105EC300E70DC3CD33CD33C933C9C833C8DEF0843E
:105ED30049F9E5F08FF0BE00E6FD7C00E9FFE8FE3E
:015EE300229C
:0E5F1500F88FF0A4FFE5F0CE88F0A42EFE2257
:10000300EF8DF0A4F9A8F0EF8CF0A428F8EE8DF0B2
:06001300A428FEE9FF2213
:105EF500600D782B025EFF007830D8FED5E0F822E1
:105F0500EEC0E07E00125E03EFFDEEFCD0E0FE2267
:0C5F3000EEC0E07E00125E03D0E0FE2216
:03001B0002001EC2
:0300530002005652
:03009B00020071EF
:03000000025F504C
:095F500075817475D000023D0456
:0B5F3C00E5822FF582E5833EF583220D
:0A0049000582D5820215831582227C
:10001E00C0E0C0F0C083C082C0D075D000123C3E9C
:0B002E00D0D0D082D083D0F0D0E032E0
:10005600C0E0C0F0C083C082C0D075D000123C4161
:10006600D0D0D082D083D0F0D0E032C0E0C0F0C093
:1000760083C082C0D075D000123CC6D0D0D082D00A
:0600860083D0F0D0E0324F
:00000001FF
